:103AC600C2AF53FFBFE4F5F18EF38FF212000AAFD7
:063AD600F443FF40D2AFF3
:013ADC0022C7
:103A9100C2AF53FFBF75F1A08EF38FF2AF058FF464
:0B3AA10012000A43FF40D2AFAFF42236
:1038A6009062AEEEF0A3EFF0C2AF53FFBF75F180AA
:1038B60012000A75F1309062AEE0FEA3E0FF8EF3CF
:0E38C6008FF2E4F5F412000A43FF40D2AF2265
:01000A0022D3
:103B4A00EEF0A3EFF0E4A3F0A3F022E0FEA3E0FF7F
:023B5A00C32284
:1037E1009061FD123B4A9061FD123B55906200E0F1
:1037F1009F9061FFE09E501A000000000000000051
:103801000000906200E004F070DC9061FFE004F0E1
:0338110080D4223E
:103846009061F9123B4A9061F9123B559061FCE098
:103856009F9061FBE09E50177FE87E031237E19050
:1038660061FCE004F070DF9061FBE004F080D72299
:103876009062A6123B4A9062A6123B559062A9E05E
:103886009F9062A8E09E50177F0A7E0012384690ED
:1038960062A9E004F070DF9062A8E004F080D7220D
:103B5C00759850438920438780758BFC758DFCD2FA
:023B6C008E22A7
:073BC100C298C299D2AC22A8
:083BB9008F993099FDC2992299
:1026DF00F090627EE03400F0906274E0FF90626EE2
:1026EF00E0FBA3E0FAA3E0F9EF1213C1906275E0EB
:1026FF0090626EFFE0FBA3E0FAA3E0F9229062097B
:10270F00E0FEE42401FFEE3440FE22EFF0A3EBF0F5
:10271F00A3EAF0A3E9F022906268E0FF90627EE006
:10272F00FCA3E0AA04F97B00220B906217EBF0A345
:10273F007462F0A37474F0A3E4F0A322FEE42411F6
:10274F00FFEE3440FEA3E0FD22900001EF1213D301
:10275F00906276E09000021213D3906277E09000BF
:10276F00031213D3906278E022906209E0FEE42412
:10277F0024FFEE3440FE22906209E0FEE42425FFA0
:10278F00EE3440FE22EFFD7C00E0FEE42DFFEC3E38
:10279F0022906209E0FEE42428FFEE3440FE2290EE
:1027AF006209E0FEE42429FFEE3440FE22E4F0A3A8
:1027BF00F0A3F0A3F02225E0249BF582E43461F529
:1027CF0083E022E0FF90627CE4F0A3EFF0E0FE22D2
:1027DF00906279E07C002400FFEC3E22900003021F
:1027EF001394906209E0FEE42404FFEE3440FE22CD
:1027FF00FFEE3440FE90628622FFEE3440FEA322AD
:10280F00E0FDA3E090621CCDF0A3EDF022E0FDA36C
:10281F00E090621ACDF0A3EDF022FEF0FCA3EFF0F2
:10282F00FD22E0F9A3E0FAA3E0906217C922E0FECF
:10283F00E42400FFEE3440FE22E0FFAA04A9059035
:10284F006219E42290000102139490000202139483
:10318600906209EFF090620BEAF0A3EBF090620A0E
:02319600EDF05A
:1031980064016018E0FF64026012EF6403600DEFE1
:1031A80064046008EF64056003023241906209E03C
:1031B800FF123A1090620912283D90620DE0FD90CE
:1031C800620AE04DFD123B0B90620BE0FCA3E04C61
:1031D800601C1227F1C006C007ECFDD007D006120C
:1031E800324C2405FFEE3440FE90620B802C906236
:1031F800B1E004F070069062B0E004F01227F1C06C
:1032080006C0079062B0E0A3FDD007D00612324C8A
:103218002405FFEE3440FE9062B0A3E0FD123B0BA4
:1032280012270C7D01123B0B12270C123A40EF704B
:10323800F790620E7401F08005E490620EF09062DF
:033248000EE0FF96
:0B324B0022123B0B906209E0FEE4221F
:103A1000906215EFF01227107D10123B0B9062158B
:103A200012270F123A40EF70F4906215E0FF7DFF0D
:033A3000023B8EC8
:05377400906209EFF076
:10377900123B20EF6413701F90620912270F7D021C
:10378900123B0B90620912270F123A40EF70F49026
:10379900620A7401F08005E490620AF090620AE01E
:0137A900FF20
:0137AA0022FC
:062C390090629812271AB8
:102C3F0012137BFFB4FF18906299122703122853C7
:102C4F00B4FF0C122859B4FF061227EBF46022EFE1
:102C5F007015906299122703122853700A1228597F
:102C6F0070051227EB600A90629CE07002A3E0707F
:102C7F0008E490629EF0022D3790629E7401F090EE
:102C8F006298E0FEE4240C12280812270312137B2B
:102C9F00122D4B240D122808122703900001122D1C
:102CAF003D240E122808122703900002122D3D24F6
:102CBF000F1228081227031227EB122D4B2410FF97
:102CCF00EE3440FEC006C00790629CE0A3FDD00723
:102CDF00D006123B0B906298E090629C12274B1229
:102CEF003B0B12392D90629812270F7D04123B0B6C
:102CFF0090629812270F123A40EF70F4122D56641B
:102D0F00156022122D566417601B906298E0FF1217
:102D1F003BB0EF30E3E6906298E0FF7D08123B8E08
:0D2D2F00E490629EF0123AF490629EE0FF84
:102D3C0022121394FD123B0B906298E0FEE422FDEC
:102D4C00123B0B906298E0FEE422906298E0FEE465
:0C2D5C002403FFEE3440FE123A40EF2248
:103AAC00906209EFF01227107D08123B0B9062090F
:0A3ABC0012270F123A40EF70F422B7
:062AFF0090620912271A83
:102B050090620F1227BCA3F0A3F0906209E0FE12B9
:102B150027C5FCA3E0FD90620DE0FAA3E0FBD39D81
:102B2500EA9C4011EE1227C5FDA3E0906213CDF09B
:102B3500A3EDF08008906213EAF0A3EBF090620930
:102B4500E0FF1235F5906211EEF0A3EFF0122C2F95
:102B55006417600EEF641C6009E4906213F0A3F043
:102B65008015906213E0FCA3E0FDC3906212E09D26
:102B7500906211E09C40C6122778123A4090620F8D
:102B8500E4F0A3EFF0122786123A40906210122764
:102B95009490620F12282990620912284812271E64
:102BA50090621312280F90620A122703122F9E902B
:102BB5006213E0FEA3E0FF906210E02FF090620F39
:102BC500E03EF0122778C006C00790620FE0A3FD33
:102BD500D007D006123B0B12278690620FA3E0FDAB
:102BE500123B0B90620912270F7D20123B0B90625E
:102BF5000912270F123A40EF70F4906209E0FF12B4
:102C05003BB0EF20E411122C2F70EF906209E0FF2A
:102C1500123A10E4FEFF22906209E0FF7D10123B9C
:092C25008E906213E0FEA3E0FFB3
:0B2C2E0022906209E0FF123B20EF2221
:0632560090620912271A24
:10325C0090620F1227BCD390620EE0940090620D26
:10326C00E0940050030233111227A0123A409062EE
:10327C000FE4F0A3EFF01227AE123A409062101256
:10328C00279490620F122829906209E0FFAA04A9E2
:10329C00057B00C002C001A312283112271E9062C8
:1032AC000D12281CD001D00212309D90620DE0FE50
:1032BC00A3E0FF906210E02FF090620FE03EF0125E
:1032CC0027A0C006C00790620FE0A3FDD007D00670
:1032DC00123B0B1227AE90620FA3E0FD123B0B903A
:1032EC00620912270F7D40123B0B90620912270FC7
:1032FC00123A40EF70F490620DE0FFA3E09062117F
:0D330C00CFF0A3EFF0906211E0FEA3E0FF10
:013319002291
:0623A00090628012271A72
:1023A600E490628B1227BD906280E01227C5FEA3DF
:1023B600E0FF906284E0FCA3E0FDD39FEC9E906278
:1023C6008B4007EEF0A3EFF08005ECF0A3EDF09064
:1023D600628612270312137B700F122853700A129B
:1023E600285970051227EB6014906289E07002A3E9
:1023F600E0600A90628BE07002A3E0700AE49062EB
:102406008BF0A3F002251A906280E0FEE4240CFF14
:10241600EE3440FE12137B122531240D1227FF12D3
:102426002703900001122523240E1227FF122703EB
:10243600900002122523240F1227FF1227031227CA
:10244600EB1225312410FFEE3440FEC006C0079083
:102456006289E0A3FDD007D006122548E090628984
:1024660012274B12254812277B123A4090628DE4C0
:10247600F0A3EFF0906280122789123A40EFFD7CBC
:102486000090628E122798FE90628D12282A906222
:102496008012284812271E90628B12280F906281A4
:1024A600122703122F9E90628BE0FEA3E0FF90623C
:1024B6008EE02FF090628DE03EF090628012277BD6
:1024C600C006C00790628DE0A3FDD007D006123B80
:1024D6000B90628012278990628DA3E0FD123B0B60
:1024E60012392D90628012270F7D20123B0B9062CD
:1024F6008012270F123A40EF70F412254F20E40F96
:1025060012254F30E3F47D1812253CE4FEFF227DB0
:0C2516001012253C90628BE0FEA3E0FF59
:1025220022121394FD123B0B906280E0FEE422FD26
:10253200123B0B906280E0FEE422906280E0FF1288
:102542003B8E123AF422123B0B9062802290628000
:07255200E0FF123BB0EF2295
:0625590090626812271ACF
:10255F00E490627C1227BDD390626DE0940090628C
:10256F006CE0940050030226CE9062681227A312EB
:10257F003A4090627EE4F0A3EFF09062681227B1C8
:10258F00123A40EFFD7C0090627F12279890627E96
:10259F00F0A3EFF090626812283D123A40EF540713
:1025AF0024FD6053146073240260030226B71227C0
:1025BF0026C0031227387408F0D0031226D7240838
:1025CF001226DF122758906271122702E48FF01241
:1025DF00146E90627112270312140BFE1227DF8FF5
:1025EF00F012146E90627A1227D290627BE0240070
:1025FF00FFEC3EA302265C122726C0031227387475
:10260F0006F0D0031226D724061226DF12275812FF
:10261F0027D31227DF90627C8033122726C0031244
:10262F0027387402F0D00312309D90627FE02402AD
:10263F00F090627EE03400F09062741227D29062C4
:10264F00751227E2CF24FECF34FF90627CF0A3EF08
:10265F00F0122726C002C00190626912283112279A
:10266F001E90627C12281CD001D00212309D906205
:10267F007CE0FEA3E0FF90627FE02FF090627EE0AF
:10268F003EF09062681227A3C006C00790627EE0FA
:10269F00A3FDD007D006123B0B9062681227B190B2
:1026AF00627EA3E0FD123B0B90626812270F7D4004
:1026BF00123B0B90626812270F123A40EF70F490A2
:0726CF00627CE0FEA3E0FFC6
:0926D6002212309D90627FE02287
:102E89003D3D3D3D3D3D3D3D3D3D3D3D3D3D3D3D69
:102E99003D3D3D3D3D3D3D3D3D3D3D3D3D3D3D3D59
:102EA9003D3D3D3D3D3D3D3D3D3D3D3D3D3D0D0AAC
:102EB9000020202020202020573731303041202089
:102EC9004E657420436F6E66696720496E666F723E
:102ED9006D6174696F6E2020202020202020200D34
:102EE9000A004D414320414444524553532049501F
:102EF900203A20252E3262782E252E3262782E2510
:102F09002E3262782E252E3262782E252E32627864
:102F19002E252E3262780D0A00252E3362752E2554
:102F29002E3362752E252E3362752E252E3362754A
:102F3900005355424E4554204D41534B20203A20D1
:102F490025730D0A00472F57204950204144445208
:102F5900455353203A2025730D0A004C4F43414CE9
:102F69002049502041444452455353203A20257367
:102F79000D0A00C0A80102C0A80101FFFFFF00005F
:102F890008DC1122330202020202020202020202D8
:052F9900020202020229
:0B3A74004861AB0000000000000000F3
:10285F00906200E025E0FF9061FFE033FE749B2F54
:10286F00F58274613EF58322906200E025E0FF90CF
:10287F0061FFE033FE748B2FF58274613EF5832286
:10288F00AC02AD03C39DFFEE9CF0A3EFF0A3E0FEFF
:10289F00A3E0FFE422F0A3E4F0747B2FF5827461D0
:1028AF003EF58322F0A3E4F0746B2FF58274613E42
:1028BF00F58322FFEE3440FEE0FBA3E0FAA3E0F93C
:1028CF008D828C83121394FD123B0B9061FFE0FC01
:1028DF00A3E0FD227D017BFF7E007F040213552FB5
:1028EF00FFE43EFEED34FEFDEC338F0F8E0E8D0DAB
:1028FF00F50C2225E024B7F582E43461F583E0FE80
:10290F00A3E0222FFFE43EFEE434FEFDE433FC227D
:10291F007D017BFF7E007F080213557A00AB07E035
:10292F00FEE422E0F510A3E0F51122EFFD7C00EBB1
:10293F00FEE42DFBEC3EFA4B228F0F8E0EF50DF5BC
:10294F000C22F583E05AFEA3E05FFBAA06E922FE04
:10295F00E42DFFEC3EF0A3EFF022F583E0FCA3E0C3
:10296F00C39FEC9E22C2AF7593FE8F828E8322EFA0
:10297F00F0E4A3F0A3F0FBFA22906209E0FEE42258
:10298F00A3E0FAA3E0FF2225E024C7F582E4346137
:10299F002225E0249BF582E434612225E0248BF587
:0529AF0082E434612206
:103ADD00123BCEC2AF123B5C75EBFF75ECFF75ED83
:073AED00FF75EEFFD2AF22CE
:101D140078317C627A2F797C1228E378357C627A78
:101D24002F79801228E378397C627D017BFF7A2F3A
:101D340079841228E7783D7C627D017BFF7A2F79D4
:101D4400887E007F0612135578437C627A2F798E41
:101D540012291F784B7C627A2F799612291F7B01F6
:101D64007A6279391239579062317F0F121F5C9071
:101D740062327F10121F5C9062337F11121F6490D5
:101D840062347F12121F649062357F01121F6C90BF
:101D940062367F02121F6C9062377F03121F7490A9
:101DA40062387F04121F74123AF490623D7F091264
:101DB4001F7C90623E7F0A121F7C90623F7F0B1251
:101DC4001F849062407F0C121F84906241E0FD7F6B
:101DD4000D7E00123B0B906242E0FD7F0E7E0012EE
:101DE4003B0B9061FC7401F0A37462F0A3744BF09C
:101DF4007B017A627943121FA4121F9A7BFF7A2E09
:101E040079BA121A1A121F9A7F097E00123A40C038
:101E1400077F0A7E00123A40C0077F0B7E00123A09
:101E240040C0077F0C7E00123A40C0077F0D7E0041
:101E3400123A40C0077F0E7E00123A40906211EFC2
:101E4400F0906210D0E0F090620FD0E0F090620E5B
:101E5400D0E0F090620DD0E0F090620CD0E0F07B26
:101E6400FF7A2E79EB121A1A7B017A62796412399D
:101E7400A390620C74FFF0A3742FF0A37422F0906B
:101E84006264E090620FF0906265E0906210F090FE
:101E94006266E0906211F0906267E0906212F07BFB
:101EA400017A627953121A1490620C7401F0A374CB
:101EB40062F0A37453F07BFF7A2F793A121A1A7FD7
:101EC400017E00123A40C0077F027E00123A40C0F1
:101ED400077F037E00123A40C0077F04121F8CD094
:101EE400E0F0906210D0E0F090620FD0E0121F3367
:101EF4007A2F794E121A1A7F0F7E00123A40C007C9
:101F04007F107E00123A40C0077F117E00123A40D3
:101F1400C0077F12121F8CD0E0F0906210D0E0F066
:0F1F240090620FD0E0121F337A2F7964021A1ADD
:101F3300F090620C74FFF0A3742FF0A37422F07B73
:101F4300017A627953121A1490620C7401F0A3742B
:101F530062F0A37453F07BFF22E0FD7E00123B0B83
:101F630022E0FD7E00123B0B22E0FD7E00123B0BC4
:101F730022E0FD7E00123B0B22E0FD7E00123B0BB4
:101F830022E0FD7E00123B0B227E00123A4090625B
:101F930012EFF0906211227BFF7A2E7989121A1ABE
:011FA300221B
:043BCE0075FF40221D
:103B6E0075FE0843FE207F647E0012384653FEDF4A
:013B7E002224
:103B0B00A2AFE433FC122974EDF0E4F593AF04EFAC
:043B1B0024FF92AF42
:013B1F002283
:0D3A3300906215E0FEE42420FFEE3440FE1A
:103A4000A2AFE433F9122974E0FFE4F593AD01ED80
:043A500024FF92AF0E
:013A5400224F
:093BB000EFFEE42402123A3B226C
:0D3B8E00EFFEE42402FFEE3440FE023B0B8C
:0B1FA4009061F9EBF0A3EAF0A3E9F074
:101FAF00E4906201F0A3F0A3F0A3F09061C77480F6
:101FBF00F0A3E4F09061B774C0F0A3E4F09061FF78
:101FCF00F0A3F01228DAFEE4241F9061F91228C260
:101FDF00FEE4241E9061FC1228C225E0FFEC1228BB
:101FEF006AE4F0A3F0122884E4F0A3F0C390620136
:101FFF00E0648094C050679061F9E0FBA3E0FAA31E
:10200F00E0F98D828C8312139424FE601D24FE60F0
:10201F002624FC602E24F86036240F704112285FAE
:10202F0074041228A4740302206812285F74081223
:10203F0028A4740702206812285F74101228A47451
:10204F000F801612285F74201228A4741F800A12A2
:10205F00285F74401228A4743FF0A374FFF0C3905C
:10206F006203E0648094C050729061FCE0FBA3E0D7
:10207F00FAA3E0F9A3E0FEA3E0FFF5828E8312132B
:10208F009424FE602224FE602B24FC603324F8602D
:10209F003B240F7046EF25E0FFEE122882740412E6
:1020AF0028B374030220E512287774081228B3743A
:1020BF00070220E512287774101228B3740F8016C8
:1020CF0012287774201228B3741F800A122877748D
:1020DF00401228B3743FF0A374FFF01228DA25E002
:1020EF00FFEC12286AE0FAA3E0FB906202E02BF00B
:1020FF00906201E03AF0122884E0FEA3E0FF9062C4
:10210F0004E02FF0906203E03EF0ED4C607B9061B5
:10211F00FFA3E025E0FFEC33FE74992FF582746185
:10212F003EF583E0FAA3E0FB74C52FF58274613EA0
:10213F0012290B2BFBEE3AFAED25E0FFEC33FE7480
:10214F00C72FF58274613EF583EAF0A3EBF0748933
:10215F002FF58274613EF583E0FCA3E0FD74B52F8B
:10216F00F58274613E12290B2DFDEE3CFC9062004E
:10217F00E025E0FF9061FFE033FE74B72FF5827426
:10218F00613EF583ECF0A3EDF0906200E004F07097
:10219F00069061FFE004F0C3906200E09408906144
:0B21AF00FFE0648094805003021FD208
:0121BA002202
:023B2000AC07F0
:103B22007BFFECFEE42403123A3BEF6B6004AB072D
:023B320080F021
:013B3400226E
:0335F500906215CC
:1035F80012297E123A3390621512292A2421123A8E
:103608003B12293A6022123A33906216E4F0A3EF93
:10361800F0906215E0FEE42421123A3BEFFD90623F
:1036280017E090621612295E906216E0FEA3E0FF92
:073638006B7002EE6A70BC2A
:01363F002268
:0335A3009062092A
:1035A60012297E1229882426123A3B906209122992
:1035B6002A2427123A3B12293A6024122988242603
:1035C600123A3B90620AE4F0A3EFF012298824270E
:1035D600123A3BEFFD90620BE090620A12295E9070
:0E35E600620AE0FEA3E0FF6B7002EE6A70B5B1
:0135F40022B4
:052F9E00906215EFF048
:102FA300AF01906220EAF0A3EFF090621912298F2B
:102FB300906215E0F925E0247BF582E4346112295F
:102FC3005112299612290B2BFFEE3A906222F0A39D
:102FD300EFF090621DE02BFF90621CE03AFEE912D5
:102FE30029A01229694003023075906215E0122965
:102FF300A012290B90621E12288FFCFDC004C0058D
:10300300C006C00712289C1228EE90621E122932B5
:10301300D007D006D005D00412348990621EE0FE9A
:10302300A3E0FF906221E02FF0906220E03EF0C326
:1030330090621DE09FFF90621CE09E90621EF0A3D1
:10304300EFF0906215E0122996F583E0FFA3E0907C
:103053006222CFF0A3EFF090622012289DFCFDC006
:1030630004C005C006C00712289C1228EE90621EF9
:10307300801990622012289DFCFDC004C005C00683
:10308300C00712289C1228EE90621C122932D00726
:09309300D006D005D004123489E6
:01309C002211
:0E309D00906213EFF0A3EBF0A3EAF0A3E9F0CA
:1030AB00A312298F906220EAF0A3EFF09062141222
:1030BB00298F906213E0F925E0246BF582E43461EB
:1030CB001229511229022BFFEE3A90621EF0A3EF48
:1030DB00F090621BE02BFF90621AE03AFEE9122996
:1030EB00AA1229695074906213E01229AA12290BB3
:1030FB0090621C12288F122912C006C00712289C3E
:10310B0012294890621C122932D007D0061234893A
:10311B0090621CE0FEA3E0FF906221E02FF0906232
:10312B0020E03EF0C390621BE09FFF90621AE09E8E
:10313B0090621CF0A3EFF0906213E0122902FF9053
:10314B00621EEEF0A3EFF0E4122912C006C00712C4
:10315B00289C12294890621C801690621E12289D92
:10316B00122912C006C00712289C12294890621A15
:0A317B00122932D007D00612348961
:013185002227
:1039570012137B9061B3F09000011213949061B43D
:10396700F09000021213949061B5F09000031213C7
:06397700949061B6F022FD
:10392D009061B3E0FD7F057E00123B0B9061B4E02A
:10393D00FD7F06123B0B9061B5E0FD7F07123B0B3F
:0A394D009061B6E0FD7F08023B0B1D
:103AF400E4FD7F05FE123B0B7F06123B0B7F071292
:073B04003B0B7F08023B0BA5
:1039A3009061B3E01213C19061B4E090000112136F
:1039B300D39061B5E09000021213D39061B6E0900A
:0539C30000030213D314
:103489008F0B8E0A8D098C08A2AFE433F51485934E
:1034990015781012149EA907AF0FAE0EAD0DAC0C26
:1034A900781012149EAB07C2AFE5111511AE10705A
:1034B9000215104E6022899378081214E18F828ECA
:1034C90083E0751200F5138B93AA13780C1214E19B
:1034D9008F828E83EAF080D1E51424FF92AF85159F
:0234E90093222C
:1029B4000D0A414343455320492F4F2050726F6401
:1029C400756374732C20496E632E0D0A4D6F646514
:1029D4006C204554482D44494F2D343820466972A3
:1029E4006D77617265205265766973696F6E202513
:1029F400782E2578206275696C643A25732040200E
:102A04002573200D0A0030382F32342F313800312D
:102A1400363A30323A3431004D4143204144445235
:102A240045535320495020202020203A20252E327F
:102A340062782E252E3262782E252E3262782E254B
:102A44002E3262782E252E3262782E252E3262782E
:102A54000D0A00252E3362752E252E3362752E2520
:102A64002E3362752E252E33627520005355424E47
:102A74004554204D41534B20202020202020203A33
:102A84002025730D0A0047617465776179204950E8
:102A94002041444452455353203A2025730D0A00E3
:102AA40049502041444452455353202020202020A3
:102AB4002020203A2025730D0A004F505431203D28
:102AC4002025632020202020004F505432203D2018
:102AD40025630D0A00495020414444524553532074
:102AE400202020203A2025730D0A0008020101014C
:0B2AF4000101010802010101010101C4
:053A7F00420000000000
:0B3B9B007D017BFF7E007F08021355B8
:033BD200C2B72255
:033BD500D2B72242
:10163C0078E97C617A2A79EF123B9B78F17C617AAC
:10164C002A79F7123B9BE4902105F0902104F012CB
:10165C003ADD9061FC7401F0A37461F0A374F1F0B5
:10166C007B017A6179E9121FA475FF28E4F59DF5D9
:10167C009E1234EB90620C7401F0A37411F0A374FD
:10168C00FFF0A3742AF0A3740AF0A374FFF0A37400
:10169C002AF0A37413F07BFF7A2979B4121A1A7FFB
:1016AC00097E00123A40C0077F0A7E00123A40C001
:1016BC00077F0B7E00123A40C0077F0C7E00123A67
:1016CC0040C0077F0D7E00123A40C0077F0E7E009F
:1016DC00123A40906211EFF0906210D0E0F09062FC
:1016EC000FD0E0F090620ED0E0F090620DD0E0F000
:1016FC0090620CD0E0F07BFF7A2A791C121A1A7FC8
:10170C00057E00123A40C0077F067E00123A40C0A8
:10171C00077F077E00123A40C0077F08121968D075
:10172C00E0F0906210D0E0F090620FD0E01218F26E
:10173C007A2A7970121A1A7F017E00123A40C00779
:10174C007F027E00123A40C0077F037E00123A40AF
:10175C00C0077F04121968D0E0F0906210D0E0F05E
:10176C0090620FD0E01218F27A2A798A121A1A7F34
:10177C000F7E00123A40C007121987C00712198F4A
:10178C00C007121958D0E0F0906210D0E0F09062CF
:10179C000FD0E012191B7A2A79A4121A1A20890484
:1017AC007F0180027F009061D7EFF07A2A79BE1218
:1017BC001997208B047F0180027F009061D7EFF096
:1017CC007A2A79CD1219979001027401F07A007B74
:1017DC00027DE17CCAE4FF120D697F011219447F7E
:1017EC00021208007F031219447F041219A37F050B
:1017FC001219A37F06120800123700902103E06033
:10180C002A14F07F017E00123846902103E0701BF1
:10181C007B017A4179321236C37B017A41793612D7
:10182C0036867B017A41793A1237AB308B33902173
:10183C0005E0702D123640121976C007121987C0B8
:10184C000712198FC007121958D0E0F0906210D00F
:10185C00E0F090620FD0E012191B7A2A79D9121A93
:10186C001A208B05E4902105F030896C902104E05E
:10187C007066123901121976C0077F107E00123A79
:10188C0040C0077F117E00123A40C0077F127E00D5
:10189C00123A40906212EFF0906211D0E0F0906238
:1018AC0010D0E0F090620FD0E0F090620C74FFF07A
:1018BC00A3742AF0A37457F07B017A6179D8121AB9
:1018CC001490620C7401F0A37461F0A374D8F07BD3
:1018DC00FF7A2A79D9121A1A3089030217D9E4909F
:0618EC002104F00217D9EF
:1018F200F090620C74FFF0A3742AF0A37457F07B8B
:10190200017A6179D8121A1490620C7401F0A374EE
:1019120061F0A374D8F07BFF22F090620C74FFF0A8
:10192200A3742AF0A37457F07B017A6179D8121A52
:101932001490620C7401F0A37461F0A374D8F07B6C
:10194200FF227A017B037DE07CCA1208007A017BC8
:10195200037DE07CCA227F127E00123A409062121E
:10196200EFF0906211227E00123A40906212EFF084
:10197200906211227B017A4179321236C37F0F7E47
:1019820000123A40227F107E00123A40227F117EDE
:1019920000123A40227BFF243090620CF0121A1A95
:0D19A200221208007A017B037DE07CCA223E
:10370000900000E07002A3E0601A90000074FFF5E2
:10371000F01213F5FEC3E5F09440EE6480948050FF
:103720001A023BD2900102E06011900000E4F0A385
:0B3730007480F0123BD5E4900102F021
:01373B00226B
:03002300023BC8D5
:063BC800309802C29832A1
:10354900906207E0FBA3E0FAA3E0F922900102747C
:1035590001F09041267482F0A3F0A3F0A3F0E4A354
:10356900F022EBF0A3EAF0A3E9F012137BFD227439
:10357900C0F074A8A3F0A37401F022904145F07B38
:10358900017A41792622900003121394FD229000BA
:0A3599000102139490000202139443
:0B373C00906207EBF0A3EAF0A3E9F0B5
:10374700E4A3F090620AE0FD2409FFE433FE9062EF
:103757000712354C8D82758300121394FD123B0BB3
:0C37670090620AE004F0E0C3940640D732
:013773002233
:1037AB0090620712356B7F017E00123B0B1235497D
:1037BB00123597FD7F027E00123B0B1235491235F5
:1037CB009DFD7F037E00123B0B12354912358F7F17
:0637DB00047E00023B0B1E
:1036860090620712356B7F057E00123B0B90620736
:1036960012354C1235977F061236B912354C123553
:1036A6009D7F071236B912354C12358F7F087E0082
:0D36B600023B0BFD7E00123B0B90620722D1
:1036C30090620712356B7F0F7E00123B0B906207EF
:1036D30012354C1235977F101236F612354C1235CF
:1036E3009D7F111236F612354C12358F7F127E00F4
:0D36F300023B0BFD7E00123B0B9062072294
:10390100123555A3F0904132123578A374AEF0A36D
:1039110074FF123562A3123578745E12357DE4129C
:0C3921003584123A559021047401F02204
:10364000123555A3F0A3F0A37408F0A374DCF0A323
:103650007411F0A37499F0A37477F0A3740AF0A323
:103660007401F0A3F0A374FBF0A374FF123562A3FE
:10367000740AF0A37401123562123584123A55901F
:0636800021057401F02297
:1034EB00123588123BA6904126E0FFB48203308B45
:1034FB00051236408024308905123901801C904119
:10350B002AE0B40106A3E06411600F90412A740114
:10351B00F0A37411123587123A557B017A41793237
:10352B001236C37B017A41793A1237AB7B017A4170
:0E353B0079361236867B017A41792C02373CB4
:103B3500AE028EFB8FFAE4FBFDFC22EBF0A3EAF06C
:053B4500A3E9F0E422F9
:1038D400E490620AF0A2AF33F0C2AF53FFBF8FF19E
:1038E400AE04AF058EF38FF2AF038FF41207FD43DE
:0C38F400FF4090620AE024FF92AFAFF4A6
:0139000022A4
:103A5500906207123B40FBFDFC7FD01238D4906288
:0F3A650007A3E0FAA3E0FF123B357FD10238D46C
:0A3BA600AF01123B357FD20238D484
:1039C800AC02AD018CFB8DFA9062A4E0FCA3E02967
:1039D800F9EA3CAD01F5FD8DFCAD07AC06E4FB7FD3
:0439E800A10238D42C
:09341B0090628FEEF0A3EFF0A324
:10342400123B40906296F0A3F0906294E0FEA3E019
:10343400FFA3E0FCA3E0FDC39FEE6480F8EC64808E
:10344400985041906290E02DFF90628FE03CCF2431
:10345400FFCF34FF8F82F583740193FF906291E074
:10346400FBA3E0FAA3E0F9906296A3E0F5828C83D3
:10347400EF1213D3906297E004F070AD906296E07F
:0434840004F080A52B
:013488002221
:10700000C2AF75FF407F717E001271D17F617E003B
:107010001271D1E4900000F0A3F0FFFE1271B77F6F
:10702000007E681271B753FFBF75F18012000A75B8
:10703000F130900000E0FEA3E0FF8EF38FF2E4F564
:10704000F412000A43FF401271AF53FFBF75F1A065
:10705000900000E0FEA3E0FF8EF38FF2E42FF582B4
:1070600074803EF583E0F5F412000A43FF4090007F
:1070700001E004F07006900000E004F0D3900001FD
:10708000E09400900000E0946840097F317E001297
:1070900071D1800C900000E05403FEA3E04E70AA72
:1070A000A2A2B392A2A2A3B392A3C3900000E094C1
:1070B0006850030270267F427E001271D1E4900076
:1070C00000F0A3F01271AFC20020003853FFBFE4FC
:1070D000F5F1900000E0FEA3E0FF8EF38FF21200C6
:1070E0000AAFF443FF40900000E0FCA3E0FDE42D74
:1070F000F58274803CF583E06F6009D2007F437EA7
:10710000001271D1900001E004F07006900000E0E0
:1071100004F0D3900001E09400900000E0946840F7
:10712000097F327E001271D1800C900000E0540380
:10713000FEA3E04E7093C200A2A2B392A2A2A4B397
:1071400092A4C3900000E0946850030270C4C2A2ED
:10715000D2A3D2A47F7A7E001271D1020000AD07C3
:10716000EDC4540FFFC3940A400BEF75F00A84E599
:10717000F02441800CEDC4540F75F00A84E5F0242E
:1071800030FFE433FE1271D1ED540FFFC3940A4077
:107190000BEF75F00A84E5F02441800BED540F7578
:1071A000F00A84E5F02430FFE433FE1271D122901E
:1071B0000000E0FEA3E0FFAB07AA06EAFF12715E43
:1071C000AF0312715E7F0D7E001271D17F0A0271D2
:0971D000D18F993099FDC299227A
:102D68000D0A4143434553204554482D44494F2DAE
:102D780034382055706C6F616420506F7274204332
:102D88006F6E6E65637465640D0A0055706C6F61D3
:102D98006420446174616772616D3A2025730D0A7D
:102DA800005374617475733D382C206C696E656CC2
:102DB800656E6774683D25303262782066756C6C84
:102DC800646174616772616D3D2530326278206399
:102DD8006F6D706172653D253032627800537461A1
:102DE8007475733D31302C206C696E656373756D35
:102DF8003D2530326278206373756D5F63616C6363
:102E08003D25303262782C2073756D3D2530326255
:102E180078200D0A006C61756E6368696E672066BC
:102E28006C61736820636F7079206F70657261746C
:102E3800696F6E2066726F6D20253034780D0A0038
:102E48000D0A666C61736820636F7079207265740F
:102E580075726E65643F213F21213F20756E65784C
:102E68007065637465642073686F756C642068614D
:102E7800766520637261736865642E2E2E2E0D0AA6
:012E88000049
:0C3A8400414146004141470041414800DB
:1021BB002406F582E43EF583E0FD7F007E80123B32
:1021CB007F9061FCE0FEA3E02407F582E43EF583FB
:1021DB00E0FD7F017E80123B7F9061FCE0FEA3E07F
:1021EB002408F582E43EF583E0FD7F027E80123BFE
:1021FB007F9061FCE0FEA3E02409F582E43EF583C9
:10220B00E0FD7F037E80123B7F9061FCE0FEA3E04C
:10221B00240AF582E43EF583E0FD7F047E80123BC9
:10222B007F9061FCE0FEA3E0240BF582E43EF58396
:10223B00E0FD7F057E80123B7F906202E0FBA3E016
:10224B00FAA3E0F974051213C1906202E0FBA3E05C
:10225B00FAA3E02274049000051213D39061F9E005
:10226B009061FCFFE0FCA3E090620DAA04F97B01F6
:10227B00E4F0A322F9900005121394904132F090F0
:10228B000006121394904133F090000712139490B0
:10229B004134F09000080213949001027401F02273
:1022AB009061F9E09061FCFFE0FCA3E0AA04F97BEC
:1022BB0001A3E0FDA3E090620DCDF0A3EDF022FAB7
:1022CB00A90790620C7401F0A3EAF0A3E9F022F9DC
:1022DB00906200E0FEA3E0FF22F9E43AFA0D023A25
:1022EB0000904150E0906200FFE0FCA3E0FDC39F33
:1022FB00EC2212137BFFFD3395E0FC906166E02D21
:10230B00F0906165E03CF022F9900005021394EE29
:10231B00F0A3EFF0D39400EE940022E0FFA3E0FAD9
:10232B00A3E0FB90620D7420F07D0122E02430F0DD
:10233B00906165E03400F022EFF0A3ECF0A3EDF038
:10234B00A3EAF0A3EBF0F922F99000010214B1F02B
:10235B00900006021394F09000070213942DFD9049
:10236B0061FCE03400FAA9057B0122F09000090220
:10237B001394F090000A021394F912137BFFC364B9
:10238B008094C122F582E43EF58322E0FF9061FC4C
:05239B00E0FCA3E022BC
:043B7F008F828E8320
:0A3B8300AF05759301EFF0E4F59330
:013B8D002215
:1039EC00FDE43EFCE92DF9EA3CFAE42FFFEE3480CD
:0439FC00FEAD07FC19
:043A00008D828C83A4
:0C3A0400759301E0FFE4F593EF0213C19D
:030800009061F90B
:100803001223439062021222D09061F9E0FF123B5F
:1008130020EF7003020D0624ED7003020D1724F779
:100823007003020CFE24056003020D1F9061F9E0C2
:08083300FF123BB0EF30E0576B
:10083B00E4906205F0906205E0FFC39407503E9090
:10084B0061F9E0FEEF6E602D906205E0FF123B2038
:10085B00BF1722E49061FEF0A3F0906205E0FF90D9
:10086B0061FCE0FCA3E0AA04F97B01E490620DF0CB
:10087B00A3F0122AFF906205E004F080B89061F9B2
:07088B00E0FF7D01123B8E2E
:100892009061F9E0FF1235A39061FE12231A500312
:1008A200020D1F9061F9E09061FC1222B2123256E1
:1008B2009061FEEEF0A3EFF01222541223531215B0
:1008C200250B05436847570AAB4368494F0ADE4385
:1008D2006849500C0843684D430B7743684E500BF0
:1008E2007743684E570B3E4368534D092744494F9F
:1008F200210A4E524144490CDE525044490C5B528B
:100902005374610CBE554461740CC25546696E093C
:10091200405741444F09605750444F096057525065
:100922004400000CDE1222A4122244F990000112AB
:1009320015015F4572729000057432020AD61222C6
:10094200A49061FCE0FEA3E01221BBF99000011229
:100952001501575F4F4B9000057406020AD612220A
:08096200A4E4906200F0A3F090
:10096A001222DB240CFDE43EFC9061FCE0FAA3E0D9
:10097A00FB2DF582EA3CF583E0F9906205F0EF245D
:10098A0006FFE43EFEEB2FF582EA3EF583E0906235
:10099A0006F0FEE95E906205F0EEF4A3F01222542E
:1009AA001222DA240C1239EC1222541222DA240C02
:1009BA0012238F121394FD906206E05DFD9062058A
:1009CA00E04DFDF0E42FFFEE3480FE123B7F122251
:0909DA00541222DA24061239EC51
:1009E300906201E004F07006906200E004F0C390AE
:1009F3006201E09406906200E09400500302096AE9
:100A03001222541223537B4F7A4479507857C312DE
:100A1300148D9062027016122247F990000112158C
:100A230001575F4F4B9000057406020AD6122257F6
:100A3300F97411122251F9900001121501525F4FFE
:100A43004B740C1222617412020CFA1222A41222A9
:100A530054F9740B122251F9900001121501525FDF
:100A63004F4B90000574061213D3E92406F9E43AB8
:100A7300FA7D007C80123A0012225424071222E4E9
:100A830012225424081222E412225424091222E4CA
:100A9300122254240A1222E4122254240B1222E4B6
:100AA300122267740C020CFA1222A4C2B69061FCE3
:100AB300E0FEA3E0FF240D12238FE0543FF5B0EFD7
:100AC3001221BBF9900001121501575F4F4B9000A3
:100AD3000574061222647406020CFA1222A412226E
:100AE3005412227F904135F012224FF990000112E7
:100AF3001501575F4F4B12225F120D20120D4B024F
:100B03000C051222A412225412231390413A1223E9
:100B13005A90413B12236190413C12229D90413DEA
:100B2300F012224FF9900001121501575F4F4B123B
:100B3300225F120D20120D55020C051222A412225F
:100B43005412231390413612235A904137122361D2
:100B530090413812229D904139F012224FF99000B2
:100B630001121501575F4F4B12225F120D2F120D09
:100B73005F020C521222A412225412227F9041359A
:100B830012237690413612237D904137F090000B6B
:100B9300121394904138F090000C12139490413941
:100BA300F090000D12139490413AF090000E12133E
:100BB3009490413BF090000F12139490413CF090BD
:100BC300001012139490413DF012224FF99000014E
:100BD300121501575F4F4B12225F120D2F12225431
:100BE3001223537B577A4E79687843C312148D705E
:100BF3000B120D4B120D5F120D55800690210374DD
:100C030064F0020C521222A41222541223139041B4
:100C13002C12235A90412D12236190412E12229DB2
:100C230090412F12237690413012237D904131F071
:100C330012224FF9900001121501575F4F4B1222F8
:100C43005F7406120D3E7B017A41792C12373C7B8F
:100C5300017A417926023A551222A4122254F974D8
:100C630024122251F9900001121501525F4F4BE4F7
:100C7300906200F0A3F01222DB7B012426F9744179
:100C83003EFA12137BFD1222542405F9E43AFAE9E1
:100C93002FF9EA3EFAED1213C1906201E004F070FD
:100CA30006906200E004F0906200E07004A3E06448
:100CB3002070C31222677425020CFA1222A4221296
:100CC30022A4122244F9900001121501575F4F4BE1
:100CD300900005E41222647406801C1222A41222DE
:100CE30054F97404122251F99000011215015F4561
:100CF30072721222677405120D3E229061F9E0FFB1
:100D0300023AAC9061F9E0FF123A109061F91223B4
:0C0D1300260231869061F9E0FF1237746F
:100D1F00227406F0122AFF9061FEEEF0A3EFF0228C
:100D2F007406F0122AFF9061FEEEF0A3EFF022F0AE
:100D3F00122AFF9061FEEEF0A3EFF0227B017A41C1
:100D4F0079321236C3227B017A41793A1237AB22BC
:0A0D5F007B017A41793612368622B4
:1033A600E490620CF0A3EB1222D21222FD12397DB8
:1033B600501990620D1222571223845005EF24D023
:1033C600800512137B24C990620CF090620EE4759E
:1033D600F0011213F590620D122257F91222FD9098
:1033E600620CE0FEC454F0F012397D501C90620D60
:1033F6001222571223845005EF24D0800512137B26
:1034060024C9FF90620CE02FF090620CE0FF9061FF
:0434160069E02FF04A
:01341A00228F
:10381400906209EB1222D29062091222572402F913
:10382400E43AFA1233A67E00C006C0079062091279
:103834002257F91233A6EFFCD0E02400FFD0E03C7D
:02384400FE2262
:030D69009061F99D
:100D6C001223439062021222D0A31222D0E4A3F0E9
:100D7C009061F9E0FF123B20EF700302123424ED76
:100D8C00700302124524F7700302120E240560034F
:100D9C0002124D9061F9E0FF123BB0EF30E0189079
:100DAC0061F9E0FF7D01123B8EE4904146F07BFF40
:100DBC007A2D7968121A1A12124E12231F5003023E
:100DCC000E60904146E070299061F9122396906272
:100DDC000D1222760412125F9061FCE0FEA3E0F586
:100DEC00828E83E0904147F09041467401F0020EF0
:100DFC0060904147E0FFD39061FFE09F9061FEE07F
:100E0C0094009061F9E0FF904146E0FD9061FDE0B7
:100E1C0050101223689061FEE0FDA3E090620DCDAE
:100E2C00800C122368904147E0FD90620DE4F0A322
:100E3C00ED12125F9061FEA3E0FF904146E02FF0AF
:100E4C00A3E0C39FF0700D904146E0906208F0E47F
:100E5C00904146F0906208E0700302120890620222
:100E6C001222571223531215250F06554461741183
:100E7C005F5546696E0E8B55706C6400001208123B
:100E8C0022A4E4904147F0A3F0A3F0906169F090A4
:100E9C006165F0A3F090414EF0A3F0906163F0A374
:100EAC00F090414CF0A3F074FF90414AF0A3F09005
:100EBC0041487401F0A312235AFE1223147C00241F
:100ECC0000FFEC3E90414EF0A3EF12229DFE122348
:100EDC00622400FFEC3E4F60069041497420F09074
:100EEC006202122257F912237EFE1223777C002411
:100EFC0000FFEC3E9061670212041222A49041485C
:100F0C00E064016003021208A3E0FF6401600302C5
:100F1C001157906205122257122313643A6008EF9E
:100F2C004402904149F022906166E0243A12233A3F
:100F3C0090000C12143664307004E5F064306008D4
:100F4C00904149E04404F022906166122337A312C9
:100F5C0023379062051222572406F9E43AFA123329
:100F6C00A6904150EFF09062051222572408F9E444
:100F7C003AFA123814906161EEF0A3EFF090415000
:100F8C00E0F92FFFE43ECF24FFCF34FFFEC39041A6
:100F9C004DE09F90414CE09E5005EEF0A3EFF09099
:100FAC00414AE0FEA3E09061611222F39E5008904A
:100FBC00414AECF0A3EDF0906208E0FD24F0FBE474
:100FCC0034FFFAE975F002A46B7003E5F06A603C3B
:100FDC00904149E04408F09061FCE0FEA3E0FF2D55
:100FEC0012238FE4F0EF2405FFE43E1222CA121202
:100FFC00797A2D79A9904150E025E090620CF0901F
:10100C006208E090620DF024F00210C7E4906200D8
:10101C00F0A3F01222EC9400503E9062051222577D
:10102C00240EF9E43AFAED25E0FFEC33FEE92FF952
:10103C00EA3EFA1233A6906200E0FCA3E02451F5DC
:10104C008274613CF583EFF0906201E004F070C3B0
:10105C00906200E004F080BB906205122257240ECF
:10106C00F9E43AFA904150E075F002A429F9EA3516
:10107C00F0FA1233A690616AEFF0906169E060407B
:10108C00904149E04410F0906208122396FD2FF530
:10109C0082E43CF583E4F0ED2405FFE43C1222CA23
:1010AC001212797A2D79E590616AE0FF90620CF06A
:1010BC00906169E0FE90620DF0EF2EA3F0021A1A17
:1010CC00906164E004F07006906163E004F090417C
:1010DC004EE0FEA3E0FF906163E0B5062AA3E0B505
:1010EC000725904149E054FEF0906165E0FEA3E0D5
:1010FC00FF906168E02FFF906167E03E4F600890C1
:10110C004149E04440F022E4906200F0A3F0122246
:10111C00EC9400400302120874512DF58274613C6A
:10112C00F583E0FF906162E02DFD906161E03CFC95
:10113C00E42DF58274803CF583EFF0906201E004BD
:10114C00F070CB906200E004F080C3904149E04421
:10115C0080F0221222A4E4904148F0A3E0906202B5
:10116C00704B122257F974041213C19062021222AE
:10117C0057F9900001121501575F4F4B9061F9E040
:10118C009061FC12226E740512126CC2AF7BFF7A56
:10119C002E791D90620C7470F0A3E4F0121A1A12DE
:1011AC0070007BFF7A2E7948121A1A80341222575B
:1011BC00F974051213C1906202122257F9900001C2
:1011CC001215015F457272904149E09000051213AF
:1011DC00D39061F9E0FF9061FC12226F7406121239
:1011EC006CE4904146F012124E12231F400E122254
:1011FC00AB1232569061FEEEF0A3EFF0E490620871
:10120C00F0229061F9E0FF1235A39061FE12231ACF
:10121C00400E1222AB1232569061FEEEF0A3EFF0AC
:10122C009061F9E0FF023AAC9061F9E0FF123A10DC
:10123C009061F91223260231869061F9E0FF123792
:01124C00742D
:10124D00229061F9E0FF1235A39061FEEEF0A3EF5D
:10125D00F022F01232569061FEEEF0A3EFF022F084
:10126D00122AFF9061FEEEF0A3EFF0227BFF7A2DA4
:08127D007993121A1A7BFF227B
:0300000002331AAE
:0C331A00787FE4F6D8FD75812102336154
:10128500E709F608DFFA8046E709F208DFFA803E4B
:1012950088828C83E709F0A3DFFA8032E309F60838
:1012A500DFFA8078E309F208DFFA807088828C83A0
:1012B500E309F0A3DFFA806489828A83E0A3F60854
:1012C500DFFA805889828A83E0A3F208DFFA804C2E
:1012D50080D280FA80C680D4806980F28033801005
:1012E50080A680EA809A80A880DA80E280CA80336E
:1012F50089828A83ECFAE493A3C8C582C8CCC583E6
:10130500CCF0A3C8C582C8CCC583CCDFE9DEE780B5
:101315000D89828A83E493A3F608DFF9ECFAA9F034
:10132500EDFB2289828A83ECFAE0A3C8C582C8CC8A
:10133500C583CCF0A3C8C582C8CCC583CCDFEADEA3
:10134500E880DB89828A83E493A3F208DFF980CC05
:1013550088F0EF60010E4E60C388F0ED2402B404FE
:101365000050B9F582EB2402B4040050AF232345A5
:0613750082239012D573E3
:10137B00BB010689828A83E0225002E722BBFE0270
:09138B00E32289828A83E49322A3
:10139400BB010CE58229F582E5833AF583E022500E
:1013A40006E92582F8E622BBFE06E92582F8E22258
:0D13B400E58229F582E5833AF583E4932272
:1013C100BB010689828A83F0225002F722BBFE010B
:0213D100F32205
:1013D300F8BB010DE58229F582E5833AF583E8F050
:1013E300225006E92582C8F622BBFE05E92582C8FC
:0213F300F222E4
:1013F500C5F0F8A3E028F0C5F0F8E5821582700283
:061405001583E038F0221F
:10140B00BB010A89828A83E0F5F0A3E022500687AC
:10141B00F009E71922BBFE07E3F5F009E31922896E
:0B142B00828A83E493F5F074019322A1
:10143600BB0110E58229F582E5833AF583E0F5F0F4
:10144600A3E0225009E92582F886F008E622BBFED1
:101456000AE92582F8E2F5F008E222E5832AF58317
:08146600E993F5F0A3E99322DC
:10146E00BB010A89828A83F0E5F0A3F0225006F7C9
:0F147E0009A7F01922BBFE06F3E5F009F31922C6
:10148D00EB9FF5F0EA9E42F0E99D42F0E89C45F0B5
:01149D00222C
:10149E00E8600FECC313FCED13FDEE13FEEF13FF2C
:0314AE00D8F12250
:1014B100BB010DE58229F582E5833AF58302156BBF
:1014C1005007E92582F802155FBBFE07E92582F87E
:1014D100021577E58229F582E5833AF583021583C2
:1014E1007401FF3395E0FEFDFC080808E6CF2FF6F6
:1014F10018E6CE3EF618E6CD3DF618E6CC3CF622CF
:10150100BB010DE58229F582E5833AF5830215AC2D
:101511005007E92582F8021593BBFE07E92582F8F9
:041521000215DD22B0
:10152500D083D082E4937012740193700DA3A393BA
:10153500F8740193F5828883E4737402936C7012D6
:101545007403936D700C7404936E70067405936F39
:0A15550060DDA3A3A3A3A3A380CA33
:1019AF00E508240CF582E43462F583E00508229003
:1019BF00620930070390620CE475F0011215F6020C
:1019CF00137B2000E97F2ED2008018EF540F249054
:1019DF00D43440D4FF30040BEF24BFB41A005003AB
:1019EF002461FFE50960021509050CE50C7002057D
:1019FF000B30070E906209E475F0011215F6EF0235
:101A0F0013C1023BB97403D2078003E4C207F50880
:101A1F0090620912160DE4F509F50BF50CE5096056
:101A2F00077F201219F280F5750AFFC201C200C2AA
:101A3F0002C203C205C206C2081219BEFF700D30E2
:101A4F0007057F00121A03AF0CAE0B22B4255FC23D
:101A5F00D5C2041219BEFF24D0B40A00501A75F073
:101A6F000A780930D50508B6FF0106C6A426F62068
:101A7F00D5047002D20380D924CFB41A00EF5004DA
:101A8F00C2E5D204021C04D20180C6D20080C0D2AB
:101A9F000280BCD2D580BAD20580B47F201219F251
:101AAF002002077401B5090040F11219AFFF121996
:101ABF00F2021A2CD208D20680951219AFFB121916
:101ACF00AFFA1219AFF94A4B700679D57A1C7BFF22
:101ADF0020022EE509602A7E008E82758300121384
:101AEF009460060EEE650A70F0C2D5EBC0E0EAC056
:101AFF00E0E9C0E0EE121C4BD0E0F9D0E0FAD0E004
:101B0F00FB12137BFF60AAEBC0E0EAC0E0E9C0E084
:101B1F001219F2D0E02401F9D0E03400FAD0E0FB42
:101B2F00E50A0460DCD50AD980877BFF7A1C7947E8
:101B3F00D202809C791080027908C206C208800800
:101B4F00D2D5790A8004790AC2D5E50A047002F564
:101B5F000AE4FAFDFEFF1219AFFC7B0820011312F5
:101B6F0019AFFD7B1030000A1219AFFE1219AFFF2B
:101B7F007B20EC3382D592D55013C3E43000069FFF
:101B8F00FFE49EFEE42001039DFDE49CFCE4CBF802
:101B9F00C201EC700CCFCECDCCE824F8F870F380F6
:101BAF0017C3EF33FFEE33FEED33FDEC33FCEB33B6
:101BBF00FB994002FB0FD8E9EB300105F8D0E0C4E8
:101BCF0048B201C0E00AEC4D4E4F78207B0070C246
:101BDF00EAB50A0040BCC0E0121C4DD0F0D0E020A6
:101BEF000104C4C0E0C4B201C0F01219DBD0F0D5BB
:101BFF00F0EB021A2C1216161AC9531B43581A9AD5
:101C0F004C1A96421B474F1B4F441B4F491AAF4369
:081C1F001B55551B39461B390A
:101C2700451B39471CF5501A9E2D1AA22E1AC52B93
:101C37001AA6231AC3201CDE2A1A5E4800001ABD02
:101C47003F3F3F00790AA2D5200314300509B91098
:101C5700020404B9080104A2D52006025001042099
:101C670002689202B509005034C0E07F20300319A2
:101C77007F30A20272067205500F121CA4C202C264
:101C870006C205C2087F30800F300503E9C0E012A5
:101C970019F2300503D0E0F9D0E0B509CC300517CB
:101CA7007F30B9100C1219F27F583004077F788003
:101CB70003B908031219F23002057F2D0219F27FCA
:101CC700202008F87F2B2006F322920280CF286E6F
:101CD700756C6C2900D2011219AF3001F8C2017876
:101CE7000930D50108F6021A5E2D504349581219DA
:101CF700AF2403B405004001E4901CF0931219E3EC
:0D1D0700743A1219E3D203750904021B435C
:10397D00EFC394414005EF94474016EFC394614067
:10398D0005EF9467400BEFC394304008EF943A5025
:06399D0003D38001C322E8
:1033260002163CE493A3F8E493A34003F68001F26B
:1033360008DFF48029E493A3F85407240CC8C333A8
:10334600C4540F4420C8834004F456800146F6DF77
:10335600E4800B0102040810204080903A74E47E59
:10336600019360BCA3FF543F30E509541FFEE4936C
:10337600A360010ECF54C025E060A840B8E493A333
:10338600FAE493A3F8E493A3C8C582C8CAC583CA5E
:10339600F0A3C8C582C8CAC583CADFE9DEE780BE16
:013A90000035
:0C155F00E6FC08E6FD08E6FE08E6FF22B8
:0C156B00E0FCA3E0FDA3E0FEA3E0FF22F3
:0C157700E2FC08E2FD08E2FE08E2FF22B0
:10158300E493FC740193FD740293FE740393FF22AE
:10159300D083D082E493F608740193F6087402931F
:0915A300F608740393F674047356
:1015AC00A8828583F0D083D0821215C31215C31282
:1015BC0015C31215C3E473E493A3C583C5F0C583A7
:1015CC00C8C582C8F0A3C583C5F0C583C8C582C889
:0115DC0022EC
:1015DD00D083D082E493F208740193F208740293DD
:0915ED00F208740393F274047314
:1015F600F8E0FBA3A3E0F925F0F0E582158270027E
:071606001583E0FA38F02221
:09160D00EBF0A3EAF0A3E9F022DE
:10161600D083D082F8E4937012740193700DA3A363
:1016260093F8740193F5828883E473740293686077
:06163600EFA3A3A380DF77
:00000001FF
